:020000040800F2
:100000008805002061200008712000087520000884
:1000100000000000000000000000000000000000E0
:10002000000000000000000000000000792000082F
:1000300000000000000000007B200008D51D000823
:10004000D31800080000000033190008FF1A000848
:10005000071F0008971F00080F2000081B2000083A
:100060000000000095200008972000089920000853
:100070009B2000089D2000089F2000080000000031
:100080005D0D00080000000000000000A120000835
:1000900000000000A3200008A5200008A7200008F9
:1000A00000000000A920000800000000AB200008AC
:1000B00010B50400002C01D1012026E03D20205C79
:1000C000002805D100203C216054200000F0DAFD1A
:1000D00002203D216054211D206800F08BFB01208F
:1000E000462160543E2160543F21605440216054B9
:1000F00041216054422160544321605444216054A2
:10010000452160543D216054002010BD70B50400AD
:100110000D00002D02D13E20205C0BE0042D02D109
:100120003F20205C06E0082D02D14020205C01E049
:100130004120205C012801D0012052E0002D04D193
:1001400002203E216054C0B211E0042D04D10220EF
:100150003F216054C0B20AE0082D04D102204021A2
:100160006054C0B203E0022041216054C0B20122B9
:100170002900206800F074FD1A482168814207D0E8
:100180002168194A914203D02168184A914201D14D
:10019000012100E00021C9B2002906D02168496C84
:1001A000802212020A4321684A642168814203D0F6
:1001B00020680F4988420DD1206880684007400FB1
:1001C0000600062E0CD0206800680121014320683B
:1001D000016005E02068006801210143206801609A
:1001E000002070BD002C0140004401400048014047
:1001F0000004004010B50400002C01D1012026E0CD
:100200003D20205C002805D100203C2160542000C6
:1002100000F039FD02203D216054211D206800F0CE
:10022000E9FA0120462160543E2160543F21605488
:100230004021605441216054422160544321605464
:1002400044216054452160543D216054002010BD7C
:10025000FEB504000D000026002D04D168463E21A5
:10026000615C01700DE0042D02D13F20205C06E0AE
:10027000082D02D14020205C01E04120205C69462D
:100280000870002D02D14220275C0BE0042D02D122
:100290004320275C06E0082D02D14420275C01E0C2
:1002A0004520275C68460078012803D13800C0B299
:1002B000012801D0012081E0002D04D102203E213F
:1002C0006054C0B211E0042D04D102203F216054DB
:1002D000C0B20AE0082D04D1022040216054C0B20F
:1002E00003E0022041216054C0B2002D04D102205D
:1002F00042216054C0B211E0042D04D102204321F8
:100300006054C0B20AE0082D04D102204421605498
:10031000C0B203E0022045216054C0B2280000288A
:1003200006D004280BD0082810D00C2815D01BE0CC
:100330002068C068022101432068C16016E020687F
:10034000C068042101432068C1600FE02068C068D4
:10035000082101432068C16008E02068C0681021BE
:1003600001432068C16001E0012006003000C0B2F6
:10037000002821D101222900206800F071FC2068AA
:100380000F49884203D020680E4988420ED1206868
:1003900080684007400F0190019806280CD0206823
:1003A0000068012101432068016005E020680068C1
:1003B00001210143206801603000C0B2FEBD000091
:1003C000002C01400004004070B5040002262068A3
:1003D0000069304000281CD02068C06830400028E8
:1003E00017D00220C04321680861012020772068CF
:1003F00080698007800F002803D0200000F0B3FC44
:1004000005E0200000F01AFD200000F018FD00209B
:100410002077042520680069284000281CD0206827
:10042000C0682840002817D00420C0432168086114
:10043000267720688069C02189000140002903D007
:10044000200000F090FC05E0200000F0F7FC200008
:1004500000F0F5FC00202077082620680069304075
:1004600000281BD02068C0683040002816D0082023
:10047000C0432168086125772068C0698007800F24
:10048000002803D0200000F06EFC05E0200000F002
:10049000D5FC200000F0D3FC00202077102021683C
:1004A0000969014000291CD02168C968084000285A
:1004B00017D01020C0432168086126772068C069E2
:1004C000C02189000140002903D0200000F04BFC2E
:1004D00005E0200000F0B2FC200000F0B0FC00209D
:1004E0002077012021680969014000290BD021688B
:1004F000C9680840002806D00120C043216808616F
:10050000200000F09DFC802021680969014000293D
:100510000BD02168C9680840002806D08020C0435D
:1005200021680861200000F08CFC402021680969E6
:10053000014000290BD02168C9680840002806D076
:100540004020C04321680861200000F07BFC20208F
:1005500021680969014000290BD02168C968084059
:10056000002806D02020C04321680861200000F048
:100570006AFC70BDF8B504000D00170000263000BD
:10058000694608703C20205C012801D102205EE011
:1005900001203C216054002F12D1EB686A68296861
:1005A000206800F08CFA206880690C21884321685B
:1005B000886120688069A96801432068816142E000
:1005C000042F13D1EB686A682968206800F0B6FA36
:1005D000206880695D4901402068816120688069E8
:1005E000A96809020143206881612CE0082F12D11B
:1005F000EB686A682968206800F0D2FA2068C06950
:100600000C2188432168C8612068C069A96801433A
:100610002068C16117E00C2F13D1EB686A68296864
:10062000206800F0DBFA2068C06948490140206872
:10063000C1612068C069A968090201432068C161DD
:1006400001E0694608703C20265468460078F2BDF7
:10065000F4B504000E0000252F003C20205C01288A
:1006600001D1022071E001203C2160540099002951
:1006700006D004291BD0082932D00C2947D05FE0CE
:100680003100206800F0EBF8206880690821014300
:10069000206881612068806904218843216888611D
:1006A00020688069316901432068816149E0310037
:1006B000206800F00CF9206880698021090101435D
:1006C000206881612068806921490140206881613A
:1006D000206880693169090201432068816130E046
:1006E0003100206800F02AF92068C0690821014320
:1006F0002068C1612068C069042188432168C861FD
:100700002068C069316901432068C16119E0310086
:10071000206800F048F92068C06980210901014380
:100720002068C1612068C069094901402068C16131
:100730002068C0693169090201432068C16100E095
:1007400007003C2025543800C0B2F2BDFFF3FFFF84
:10075000FFFBFFFF70B504000E003C20205C012869
:1007600001D1022024E001253C20255402203D2116
:1007700060543100200000F04BF9002806D03D20E5
:10078000255400203C216054012011E02068C068FD
:10079000402188432168C8602068C068054901403D
:1007A0002068C1603D20255400203C216054002079
:1007B00070BD0000FFBFFFFF00B5020000200B006E
:1007C000002B06D0042B08D0082B0AD00C2B0CD001
:1007D0000FE013685B6B18000BE013689B6B18004D
:1007E00007E01368DB6B180003E013681B6C18004C
:1007F000FFE700BD10B503687F4A904202D07F4CEE
:10080000A04204D17024A3431C004B6823439042B0
:100810000BD07A4CA04208D0794CA04205D0794C3C
:10082000A04202D0784CA04203D1784C1C40CB6847
:1008300023438024A3434C691C4304608B68C36238
:100840000B688362904205D06E4A904202D06E4A95
:10085000904201D10A6902630122426110BD70B564
:10086000026A01239A430262056A4368846970221E
:100870009443032294430A6822430224A5438C68CC
:100880002C435D4DA84205D05E4EB04202D05E4E74
:10089000B04206D10826B4432600CC68344304266F
:1008A000B443A84205D0574DA84202D0564DA842A5
:1008B00007D1974D1D40C84B2B404D691D438B6997
:1008C0002B43436082614D684563046270BD70B51F
:1008D000026A10239A430262036A426884698D4D5A
:1008E00025404A4E2E400C68240234432025AB4359
:1008F0008D682D011D43404B984207D18026B5439A
:100900002E00CD682D0135434026B543984205D0D1
:100910003C4B984202D03C4B984209D19F4B13402C
:10092000BD4A1A404B699B0013438A6992001A43DF
:10093000426084614B688363056270BDF0B5026AF2
:10094000734B13400362046A4268C56970239D4378
:1009500003239D430B682B439F4D25408C68240245
:100960002C43254DA84206D1AB4E2640CC68270229
:1009700037438A4C3C40A84205D0224DA84202D0C1
:10098000214DA84209D1AB4D1540AB4A2A404D69D3
:100990002D0115438A6912012A434260C3614D68E3
:1009A000C5630462F0BD70B5026AA24B13400362D6
:1009B000036A4268C469574D2540144E2E400C68A6
:1009C000240234439C4D1D408B681B032B430A4D6E
:1009D000A84205D00B4DA84202D00B4DA84204D12D
:1009E000964D15404A6992012A434260C4614D68A0
:1009F0000564036270BD0000002C0140000400404B
:100A0000002000400044014000480140FFFCFFFF7F
:100A1000FEB505000C000026286880687021884318
:100A2000616801430720814327680F432868876076
:100A3000606800283DD010283BD0202839D03028CD
:100A400037D040280CD0502827D060282BD07028D1
:100A500030D12369A268E168286800F0DFF82BE054
:100A60002068052801D1012028E02868006A00904C
:100A70002868006A0121884329680862286880691B
:100A8000F0218843216909010143019101982968F6
:100A900088610098296808620EE02269A1682868C8
:100AA00000F03AF808E02269A168286800F062F8CE
:100AB00002E001E0012006003000C0B2FEBDF0B54A
:100AC000046A0125AC4304628669056A5C4CA04255
:100AD00002D05C4CA04201D1012400E00024E4B229
:100AE000002C03D00324A643164302E00124344320
:100AF0002600F024A6431F01F0243C4034430A267C
:100B0000B5430A260E402E4384610662F0BD000004
:100B1000FFFEFFFFFF8FFFFF30B4036A046A012569
:100B2000AC4304628469F025AC43150125430A24D3
:100B3000A3430B438561036230BC7047F0B4046A81
:100B40001025AC4304628569046A3F4E2E401702AB
:100B500037433E4D3D401F03F02636023E402E43B4
:100B6000A025AC430F01A0253D40254386610562C9
:100B7000F0BC704730B4036A1024A3430362846955
:100B8000036A324D254014032C43A025AB430D01CD
:100B90001D438461056230BC70470000FFFBFFFF0E
:100BA000F0B4046A2A4D25400562C669056A03242B
:100BB000A6431643F024A6431F01F0243C403443CF
:100BC000244E2E400F02A0252D013D403543C46127
:100BD0000562F0BC70470000FFFDFFFFF0B4046A3F
:100BE000144D25400562C469056A174E264014025B
:100BF0003443164E26401F03F02424023C40344365
:100C0000154E2E400F03A0252D023D403543C461F3
:100C10000562F0BC70470000FFF7FFFF70B4846806
:100C20000E4D254016000E431C0234432C438460B5
:100C300070BC7047FFEFFFFFFFDFFFFFFFBFFFFF4D
:100C4000002C014000040040FFFCFFFFFF0FFFFFEE
:100C5000FFFEFFFFFFF5FFFFFF5FFFFFFF00FFFF4E
:100C600070B41F2301240D001D40AC40056AA5434C
:100C70000562056A0E00334016009E402E43066250
:100C800070BC704770477047F8B586B0802080020E
:100C90005A490A6802430A600968084000900098AF
:100CA00002275748016839430160006838400090C6
:100CB00000984020019002970120039003200490A7
:100CC0000120059001A99020C00500F0BDF8012287
:100CD0000021102000F03FFA102000F046FA494CA5
:100CE000494E00F086FD494900F09CFD2100401866
:100CF0003080474D47482860EC60308868600024A9
:100D00002C61AC606C61AC612800FFF773FA424E55
:100D1000B460F4603460012070600022310028006B
:100D2000FFF728FC37607760042231002800FFF7C6
:100D300021FC3A4904200860502048608C60CC6057
:100D40000C612800FFF706FD00212800FFF780FA5C
:100D500004212800FFF77CFA07B0F0BD80B52C48CD
:100D6000FFF732FB01BD38B50400207F012835D1E3
:100D70002B4D00212000FFF71FFD28602868002868
:100D800027D02248296800F04DFD27490860254DED
:100D900004212000FFF710FD2860286823498842BD
:100DA00004D323480178491C017005E000200100AC
:100DB000204A11701E4908701D48007810280DD176
:100DC0001C480178002909D1012101701A480170DD
:100DD00004E00020134908601349086031BD00B5E4
:100DE00015480078002801D0012000E00020C0B2A2
:100DF00000BD114908707047000000001410024047
:100E00001C100240FFFF00007801002040420F004C
:100E10008400002000040040540100203001002024
:100E200064010020680100206C01002041060000E0
:100E300081010020800100207F0100207047704761
:100E40007047704770477047F1B582B0002308685B
:100E5000D840002800D1F3E00124086825009D4017
:100E6000054001950198002800D1E7E00325486876
:100E70002840012803D04868284002281ED1029843
:100E800086681F00022047432800B8408643CF6889
:100E9000BC461800022778436746874037430298CC
:100EA0008760029846682000984086434868000999
:100EB0002040984030430200029842604868284031
:100EC000032812D00298C6681F000220474328005A
:100ED000B84086438F68BC461800022778436746AF
:100EE000874037433A000298C26048682840022889
:100EF00021D10298DE0804277E438019076A072063
:100F000000970F26B4461F00074004267743664625
:100F1000BE40009FB743BC460E691F0038400427FF
:100F20007843864067463E4332000298DE08042735
:100F30007E4380190262029806681F000220474320
:100F40002800B84086434F682F40BC46180002274F
:100F500078436746874037433A0002980260486802
:100F6000C026B6020640002E68D03C4806682643DC
:100F700006600068204000900098394E98080427C9
:100F80007843305800900F27BC461F002800384097
:100F900004277843674687400098B843009002983A
:100FA0009027FF05B84201D1002410E002982D4A95
:100FB00090420CD002982C4A904201D1022406E0C3
:100FC00002982A4A904201D12C0000E005240098A2
:100FD0001A00154004225543AC40044398080422EB
:100FE00050433450224A1068019DA8434D68ED02D9
:100FF00002D504000198204310601E4C2268019D18
:10100000AA434D68AD0202D51000019A0243226046
:10101000194C2068019DA8434D68AD0302D502001C
:10102000019810432060154C2268019DAA434D6829
:10103000ED0302D51000019A024322605B1C06E713
:10104000F7BD00B51300DBB2002B03D00B009BB241
:10105000836102E00B009BB2836200BD1810024066
:10106000080001400004004800080048000C004847
:10107000080401400C040140040401400004014044
:1010800000B5010049B2002905D40121C206D20EE3
:1010900091403C4A116000BDF0B5020052B2002AF6
:1010A0001CD40322384B040064B2A40804256C430A
:1010B0001C59FF251600064008277E43B540AC4367
:1010C0008D01EDB20240082672439540254302008F
:1010D00052B29208042462439D5022E00F242B4A0E
:1010E000032305006DB22540083DAD080426754375
:1010F000060076B23440083CA4080426744316590E
:10110000FF27BC461C00044008277C436746A740D5
:10111000BE438C01E4B2034008277B439C40344328
:101120005451F0BD10B50400601E8021490488426E
:1011300001D301200EE0601E154908600321002044
:10114000C043FFF7A9FF0020124908600720124999
:101150000860002010BD70B505000C0016002100CD
:10116000280040B2FFF798FF70BD10B504002000C2
:1011700040B2FFF785FF10BD10B504002000FFF757
:10118000D1FF10BD00E100E000E400E01CED00E054
:1011900014E000E018E000E010E000E0F8B584B0F2
:1011A0000400002C01D101204AE22078C00766D556
:1011B0000C20B4490A680240042A09D00A68104089
:1011C00008280ED18020400209680140814208D1E0
:1011D000AD480068800352D5606800284FD10120D7
:1011E0002EE26068012806D1A748016880225202D9
:1011F0000A43026024E06068002809D1A24801681F
:10120000A24A0A4002600168A14A0A40026017E04F
:10121000606805280BD19C4801688022D2020A43ED
:1012200002600168802252020A43026008E0964888
:101230000168964A0A4002600168954A0A400260C5
:10124000606800280DD000F045FB05008E4800685E
:10125000800314D400F03EFB401B6528F6D3032026
:10126000EEE100F037FB050087480068800306D5F3
:1012700000F030FB401B6528F6D30320E0E1022696
:101280002068304000284FD00C207E490A68024078
:10129000002A06D00A681040082814D10868C00344
:1012A00011D4794801683140002904D0E16801294E
:1012B00001D00120C4E10168F82291432269D200E3
:1012C0000A43026030E0E06800281AD06E4F3868A8
:1012D00001210143396000F0FDFA05003868304013
:1012E000002806D100F0F6FA401B0328F6D30320AD
:1012F000A6E13868F82188432169C90001433960B3
:1013000012E0614F386801218843386000F0E2FA4A
:10131000050038683040002806D000F0DBFA401B9A
:101320000328F6D303208BE12078000728D5E06955
:10133000002812D0C34F386801210143396000F002
:10134000C9FA050038683040002819D100F0C2FA07
:10135000401B0328F6D3032072E1BA4F38680121FD
:101360008843386000F0B6FA05003868304000283D
:1013700006D000F0AFFA401B0328F6D303205FE14C
:10138000042720683840002800D18CE000206946FE
:10139000087080204005AC490968014000290AD145
:1013A000A9490A6802430A60096808400390039843
:1013B000012069460870A5480068C00514D4A348F8
:1013C0000068802149000143A048016000F082FAD2
:1013D00005009E480068C00506D400F07BFA401B5B
:1013E0006528F6D303202BE1A068012805D1984891
:1013F000016801220A43026021E0A068002809D1A7
:1014000093480168012291430160016804229143DD
:10141000016014E0A068052808D18D4801683943AF
:101420000160016801220A43026008E088480168FF
:101430000122914301600168042291430160A06888
:1014400000280FD000F046FA0500814800683040BF
:1014500000281FD100F03EFA401B7E498842F4D399
:101460000320EDE000F036FA0500794800683040CE
:1014700000280FD000F02EFA401B76498842F4D3A2
:101480000320DDE00410024000100240FFFFFEFFD9
:10149000FFFFFBFF68460078012804D16A48016815
:1014A0006D4A0A4002602078C00650D56069012864
:1014B00022D1B44800680743B2480760B1480068C9
:1014C00001210143AF48016000F004FA0500AD4876
:1014D00000683040002806D100F0FCF9401B0328CA
:1014E000F5D30320ACE0A7480168F8229143A26934
:1014F000D2000A4302602AE00421C943606988429D
:101500000BD1A0480268114001600168F8229143A4
:10151000A269D2000A43026019E09A4800680743B2
:1015200098480760974800680121884395490860FA
:1015300000F0D0F90500934800683040002806D03C
:1015400000F0C8F9401B0328F5D3032078E0206A97
:10155000002874D08C4800680C21014008294DD027
:10156000206A022838D1894F38688949014039609A
:1015700000F0B0F900908026B604386830400028AA
:1015800007D000F0A7F90099401A0328F3D30320ED
:1015900056E0994801680F229143E26A0A430260CB
:1015A000794801687B4A0A40A16A1143626A0A438A
:1015B00002603868802149040143396000F08AF9EB
:1015C000050038683040002839D100F083F9401B0D
:1015D0000328F6D3032033E06C4E30686C49014099
:1015E000316000F077F905003068800127D500F000
:1015F00071F9401B0328F7D3032021E0206A01285A
:1016000001D101201CE06048006801907A48006820
:1016100002900198802149020840616A88420CD1F9
:1016200002980007000FE16A884206D10198F02174
:1016300089030140A06A814201D0012000E000201E
:1016400005B0F0BD241002401C10024000700040A4
:101650002010024089130000FFFFFFEFF3B581B0B7
:101660000400002C01D101208BE00125634E30687D
:101670002840029988420CD230680121884302999F
:1016800001433160306828400299884201D001202E
:1016900077E002202168014000290FD02178490716
:1016A00005D539490A68E023DB0013430B6036494E
:1016B0000A68F0239A43A36813430B60216829400A
:1016C000002932D06168012905D1304800688003C3
:1016D00011D4012055E06168022905D12B4800682A
:1016E000800108D401204CE02849096808400028FE
:1016F00001D1012045E0244F386803218843616807
:101700000143396000F0E6F8009038680C21014090
:1017100060688000814208D000F0DCF80099401A2F
:1017200037498842F1D303202BE0029831682940E1
:1017300088420CD23068012188430299014331600C
:10174000306805400298854201D0012019E02078D8
:10175000400706D50C4801682A4A0A40E16811434F
:10176000016000F019F82849074A126812091207A7
:10177000120F895CC84025490860002000F0B0F8CD
:101780000020FEBD34100240041002400010024050
:10179000FFFFFFFEFFFFC2FFF8B50024200000940A
:1017A000250026001A490F680C213940042902D06F
:1017B000082902D01BE017481AE00F201649BA0C7E
:1017C0000240895C0E0015490B4A12681040085C03
:1017D0000090F80306D50F48009900F023F87043F5
:1017E000050002E00E4870430500280000E00948AB
:1017F000F2BD0648006870472C10024000200240ED
:1018000089130000FFF8FFFF5020000804000020AB
:101810000410024000127A00302000084020000826
:1018200000093D000022030A8B420BD203098B42C0
:1018300019D243088B422ED2411A00D2014652419E
:1018400010467047FF2209023FD012068B4205D393
:10185000121209028B4201D31212090203098B42B0
:1018600019D300E0090AC3098B4201D3CB01C01A86
:10187000524183098B4201D38B01C01A5241430963
:101880008B4201D34B01C01A524103098B4201D351
:101890000B01C01A5241C3088B4201D3CB00C01ABE
:1018A000524183088B4201D38B00C01A5241430836
:1018B0008B4201D34B00C01A5241884200D3401AD8
:1018C0005241CFD201461046704708B500F030F8BB
:1018D00008BDFEE701480068704700BF70010020A6
:1018E00010B50400FA2080000E490978FFF79AFF2E
:1018F00001000D480068FFF795FFFFF73DFC002849
:1019000001D001200CE0042C09D20022210000208B
:10191000C043FFF720FC05480460002000E00120E0
:1019200010BD00BF080000200400002000000020BF
:101930007047FEE770B586B014220021684600F0BB
:10194000ADF88020800251490A6802430A600A68A3
:101950001040059005988020C0020A6802430A6082
:10196000096808400590059880256D0100950120C3
:10197000019002200290032003909024E405694620
:101980002000FFF761FA009569462000FFF75CFA36
:101990001A2000903E4E69463000FFF755FA0420A9
:1019A000009069462000FFF74FFA01220421200031
:1019B000FFF747FB002229002000FFF742FB00222F
:1019C0001A213000FFF73DFB06B070BD38B50500A9
:1019D0002800C0B2012834D12E4C20782E4908703E
:1019E0002078002805D0022811D008D3032814D06D
:1019F00019E0012202212648FFF723FB13E0012210
:101A0000802149019020C005FFF71BFB0BE001225C
:101A100010211F48FFF715FB05E0012208211C4893
:101A2000FFF70FFBFFE72800C0B201282DD1207877
:101A3000032802D10020207027E02078401C20706D
:101A400023E015480078002805D0022811D008D3DB
:101A5000032814D019E0002202210D48FFF7F1FA03
:101A600013E00022802149019020C005FFF7E9FA28
:101A70000BE0002210210648FFF7E3FA05E0002200
:101A800008210348FFF7DDFAFFE731BD14100240DB
:101A9000000400487C0100207D01002010B50400F6
:101AA000080011000200200000F002F8200010BD24
:101AB0001206130A1A43130C1A4300BF094205D039
:101AC000830705D00270401C491EF9D17047000001
:101AD0001300103906D330B41400150010393CC07F
:101AE000FCD230BC490700D30CC000D504C089002B
:101AF00002D30280801C002900D502707047FEE7E7
:101B0000F8B586B08020800239490A6802430A602D
:101B100009680840009000988020000135490A6853
:101B200002430A6009680840009000980220029071
:101B300001210391032104910590C020C000019070
:101B400001A99020C005FFF77FF92B4DFFF751FE4B
:101B50002A49FFF767FE401E2880294C294820604B
:101B6000288860602848E06000262661A6606661DB
:101B7000A6612000FEF79CFA244D60202860AE602C
:101B80002E61EE60AE616E612F1DC226F6003E60D2
:101B9000042229002000FEF75BFD3E600822290098
:101BA0002000FEF755FD04212000FEF7AFFA0821C2
:101BB0002000FEF7ABFA07B0F0BD00B50200D2B2CC
:101BC000012A02D0022A05D009E00A0092B2104B85
:101BD0001A6004E00A0092B20E4B1A60FFE700BDE3
:101BE000C220C0000A4908600A4908607047000026
:101BF00014100240181002407A01002040420F00E9
:101C0000CC000020002C0140204E000014010020D8
:101C1000382C01403C2C014070B53C4C200000F0B9
:101C2000B6F8FFF7DCF800282CD00120FFF7CEFE35
:101C30009026F605002204213000FFF702FAFA256B
:101C40006D00280000F0B0F8200000F0A0F801229C
:101C500004213000FFF7F5F9280000F0A5F8200076
:101C600000F095F800F00FF8280000F09DF8200033
:101C700000F08DF80020FFF7A9FEFFF7B1FF00206C
:101C8000FFF7B7F870BD10B5214C2078002805D0BB
:101C900002280DD007D303280FD013E01D490120DF
:101CA000FFF78BFF0EE01B490220FFF786FF09E0DC
:101CB00019490120FFF781FF04E017490220FFF7CF
:101CC0007CFFFFE72078032802D10020207002E08B
:101CD0002078401C207010BD80B58CB0082000908A
:101CE00000200890012007906846FFF757FA074840
:101CF0000A49016020214160FA2189008160084978
:101D0000C16000F00FF80DB000BD000044010020DC
:101D10007E010020140500003A070000003000405A
:101D2000FF0F000070B50400002C01D101202DE050
:101D30001A48216808601A482168086060682168AC
:101D40004860A06821688860FFF7C4FD0500072689
:101D50002068C068304000280BD0FFF7BBFD401B57
:101D60002828F4D32068C0680640002EEFD0032056
:101D70000CE020680069E168884203D0E0682168CF
:101D8000086102E0074821680860002070BD01007A
:101D900004480A681060002070470000CCCC0000A6
:101DA00055550000AAAA000070B50400FFF792FD87
:101DB000050026000020C043864202D00448007877
:101DC0003618FFF787FD401BB042FAD370BD00BF45
:101DD0000800002080B500F045F800F032F81E48F9
:101DE0000178491C017001780A2901D10021017094
:101DF00000200A2824DA19490C2242438A18127A50
:101E0000002A1BD00C2242438A189288521E0C23AF
:101E10004343CB189A800C2242438A189288002AA6
:101E20000CD10C2242438A18D2880C234343CB188E
:101E30009A8001220C234343C9184A72401CD8E7F8
:101E400001BD00B506480168002902D00168491E9D
:101E5000016000BD00000000820100200C00002095
:101E60007401002003480168034A12788918016050
:101E7000704700BF700100200800002080B500F00E
:101E800043F800F00BF8FFF755FDFFF739FEFEF7BA
:101E9000FBFEFFF721FFFFF7BFFEFCE738B590B070
:101EA0003022002104A8FFF7F9FD10220021684626
:101EB000FFF7F4FD122004900120079009901020F4
:101EC00008900A9002240C9400250D95A020800310
:101ED0000E900F9504A8FFF761F9002801D000F0DB
:101EE0000FF80720009001940295039501216846A0
:101EF000FFF7B4FB002801D000F002F811B030BDAC
:101F000000B572B6FEE7FEE780B50648016810220C
:101F10000A4302600020FFF7E3FC00F005F8002010
:101F200002BD000000200240704770B4012300246D
:101F300013E00168001D194202D04D466D1E49197B
:101F40000C60091D121F042AFAD20D00960701D554
:101F50000C80AD1C1A4000D02C700268001D002AB5
:101F6000E7D170BC704730B401220EE00368C3189B
:101F700044680830144202D04D466D1E64191D6835
:101F800025601B1D241D091FF9D10168001D0029B2
:101F9000ECD130BC7047FEE710B5074979441831E1
:101FA000064C7C44163404E0081D0A6889188847EA
:101FB0000100A142F8D110BD080000002800000077
:101FC0006BFFFFFF780100000C0000200000000004
:101FD00097FFFFFF0C000000B00000000000002091
:101FE0000000000000F00DF8002801D0FFF7D4FF3A
:101FF00000BF00BF002000BF00BFFFF73FFF00F0A1
:1020000002F80120704780B500F002F801BDFEE73C
:102010000746384600F002F8FBE7FEE780B500BF50
:1020200000BF024A11001820ABBEFBE726000200E9
:1020300002030405060708090A0B0C0D0E0F101009
:102040000102030405060708090A0B0C0D0E0F1008
:102050000000000000000000010203040607080958
:102060000148804701480047AD2000087D20000856
:1020700000B5FEE700B5FEE77047704700BF00BF40
:1020800000BF00BFFFF7AEFF0400000000127A009F
:1020900001000000FEE7FEE7FEE7FEE7FEE7FEE7E1
:0E20A000FEE7FEE7FEE7FEE7FEE7FEE770471D
:040000050800207D52
:00000001FF
